:020000040800F2
:10000000400900202502000851330008533300083E
:10001000573300085B3300085F330008000000001E
:100020000000000000000000000000006333000832
:100030006533000800000000673300083D02000837
:100040003F0200083F0200083F0200083F0200088C
:100050003F0200083F0200083F0200083F0200087C
:100060003F0200083F0200083F0200083F0200086C
:100070003F0200083F0200083F0200083F0200085C
:100080003F0200083F0200083F0200083F0200084C
:100090003F0200083F0200083F0200083F0200083C
:1000A0003F0200083F0200083F0200083F0200082C
:1000B000212700083F020008092700083F02000826
:1000C0003F0200083F0200083F0200083F0200080C
:1000D0003F020008ED200008113200083F0200082E
:1000E0003F0200083F0200083F0200083F020008EC
:1000F0003F0200083F0200083F0200083F020008DC
:100100003F0200083F0200083F0200083F020008CB
:100110003F0200083F020008CD2E00083F02000801
:100120003F0200083F0200083F0200083F020008AB
:1001300000F002F800F067F80AA090E8000C824492
:100140008344AAF10107DA4501D100F05CF8AFF26F
:10015000090EBAE80F0013F0010F18BFFB1A43F0A5
:1001600001031847E4510000045200000A444FF014
:10017000000C10F8013B13F0070408BF10F8014B06
:100180001D1108BF10F8015B641E05D010F8016B4B
:10019000641E01F8016BF9D113F0080F1EBF10F8AF
:1001A000014BAD1C0C1B09D16D1E58BF01F801CBD2
:1001B000FAD505E014F8016B01F8016B6D1EF9D555
:1001C0009142D6D37047000000230024002500266A
:1001D000103A28BF78C1FBD8520728BF30C148BFAA
:1001E0000B607047662904F05684002070471FB5E5
:1001F00003F0AAFB04000020002104F0EDF8E06009
:100200001FBD10B510BD03F09BFC1146FFF7EFFFBB
:1002100003F02CF803F0B9FC03B4FFF7F2FF03BCC2
:1002200003F0FCFC0948804709480047FEE7FEE769
:10023000FEE7FEE7FEE7FEE7FEE7FEE7FEE7FEE796
:1002400004480549054A064B70470000430300086F
:100250003101000840030020400900204005002033
:10026000400500200CB50020019000906C4800680B
:1002700040F480306A49086000BF6948006800F4B3
:10028000003000900198401C0190009818B9019826
:10029000B0F5A06FF1D16248006800F4003010B1F1
:1002A0000120009001E0002000900098012843D137
:1002B0005C48006840F010005A4908600846006831
:1002C00020F0030008600846006840F00200086063
:1002D00053484068524948600846406848600846AC
:1002E000406840F4806048600846406820F47C1014
:1002F00048600846406840F4E810486008460068D6
:1003000040F08070086000BF4548006800F0007051
:100310000028F9D04248406820F003004049486076
:100320000846406840F00200486000BF3C48406812
:1003300000F00C000828F9D10CBD10B5FFF792FFB2
:1003400010BD10B53648006840F00100344908601F
:10035000084640683449084031494860084600680A
:10036000324908402E4908600846006820F4802081
:1003700008600846406820F4FE0048604FF41F0003
:100380008860FFF7DAFF4FF000602949086010BD70
:1003900010B5002100200022214B5B6803F00C0106
:1003A00021B1042906D0082928D107E0214B224C8D
:1003B000236027E01F4B204C236023E0184B5B6831
:1003C00003F47010164B5B6803F48032022303EBD6
:1003D000904022B9194B4343174C23600DE0104B5A
:1003E0005B6803F4003323B1144B4343124C236086
:1003F00003E0104B4343104C236003E00D4B0E4CC5
:10040000236000BF00BF064B5B68C3F303130C4CB3
:10041000E15C094B1B68CB40074C236010BD00001A
:1004200000100240002002400000FFF8FFFFF6FE2F
:1004300008ED00E000127A000000002000093D00F5
:100440000400002031490143314A1160704770B502
:10045000002100230F22C47804B32D4C246804F437
:10046000E064C4F5E064210AC1F10403CA404478A1
:1004700004FA03F18478144021430901254C0678DD
:10048000A155047804F01F050124AC4005786D11D6
:10049000AD0005F1E025C5F8004109E0047804F05D
:1004A0001F050124AC401C4D0678761145F8264006
:1004B00070BD1A4A0A400243154B1B1F1A60704751
:1004C00039B1134A121D12680243114B1B1D1A60E9
:1004D00006E00F4A121D126882430D4B1B1D1A6065
:1004E0007047042808D14FF0E021096941F0040168
:1004F0004FF0E022116107E04FF0E021096921F09F
:1005000004014FF0E0221161704700000000FA057D
:100510000CED00E000E400E080E100E080FFFF1F60
:1005200010B50446CC48844208D10121042000F0D3
:100530002DFB0021042000F029FB46E0C74884423F
:1005400008D10121082000F021FB0021082000F043
:100550001DFB3AE0C248844208D10121102000F07E
:1005600015FB0021102000F011FB2EE0BD48844255
:1005700008D10121202000F009FB0021202000F0FB
:1005800005FB22E0B848844208D10121402000F058
:10059000FDFA0021402000F0F9FA16E0B348844249
:1005A00008D10121802000F0F1FA0021802000F024
:1005B000EDFA0AE0AE48844207D10121801500F02F
:1005C000E5FA0021A01500F0E1FA10BD10B50121F7
:1005D000084600F0DBFA0021012000F0D7FA10BD38
:1005E0002DE9F041024600250026002000230024CA
:1005F000002791F803C00CF00F0591F803C00CF030
:10060000100CBCF1000F03D091F802C04CEA0505B4
:1006100091F800C0BCF1000F31D0146800202BE02D
:100620004FF0010C0CFA00F3B1F800C00CEA03061D
:100630009E4220D183004FF00F0C0CFA03F7BC430D
:1006400005FA03FC4CEA040491F803C0BCF1280F3E
:1006500006D14FF0010C0CFA00FCC2F814C00AE0FD
:1006600091F803C0BCF1480F05D14FF0010C0CFA12
:1006700000FCC2F810C0401C0828D1D31460B1F8A7
:1006800000C0BCF1FF0F34DD546800202EE000F103
:10069000080C4FF0010808FA0CF3B1F800C00CEA9E
:1006A00003069E4221D183004FF00F0C0CFA03F792
:1006B000BC4305FA03FC4CEA040491F803C0BCF106
:1006C000280F05D100F1080C08FA0CF8C2F81480C4
:1006D00091F803C0BCF1480F07D100F1080C4FF0AE
:1006E000010808FA0CF8C2F81080401C0828CED384
:1006F0005460BDE8F0814FF6FF71018002218170E6
:100700000421C17070470246002093680B400BB172
:10071000012000E0002070470146886880B27047E1
:1007200002460020D3680B400BB1012000E00020FE
:1007300070470146C86880B27047016170474161E7
:1007400070470AB1016100E041617047C1607047C4
:100750004FF480320A4382618161826182698269D9
:10076000704702460020434B18684FF680731840CC
:1007700040EA021008433F4B186070473E49C86189
:100780007047F0B50A46002300240021002500F040
:100790000046B6F1004F02D1364EF16901E0354E08
:1007A0007168C0F3034583B200F44016B6F5401FEC
:1007B00008D121F070612F4E766826F070662D4FBB
:1007C0007E6012E000F48016B6F5801F06D1032685
:1007D00006FA05F4A14341F0706106E0460D3601CA
:1007E00003FA06F6B14341F0706122B1460D3601BD
:1007F00003FA06F6314300F00046B6F1004F02D18D
:100800001C4EF16101E01B4E7160F0BD30B500225D
:100810008B071C0F0F2303FA04F2164B08338C10BE
:1008200053F824309343134C08348D1044F825308A
:1008300023468C1053F824308C07240F00FA04F45C
:1008400023430C4C08348D1044F8253030BD0A4940
:10085000DC3108607047000000080140000C0140D6
:10086000001001400014014000180140001C01402C
:10087000002001400000014000002042DF480068E5
:1008800040F00100DD49086008464068DC49084046
:10089000DA49486008460068DA490840D7490860E4
:1008A0000846006820F4802008600846406820F46C
:1008B000FE0048604FF41F0088607047CF49096808
:1008C00021F48031CD4A11601146096821F480215C
:1008D0001160B0F5803F03D0B0F5802F0ED106E057
:1008E000C649096841F48031C44A116007E0C34930
:1008F000096841F4A021C14A116000E000BF00BFB7
:10090000704710B501460022002300204A11012A39
:1009100002D1BA4C236806E0022A02D1B74C236AFE
:1009200001E0B64C636A01F01F02012494401C40B0
:100930000CB1012000E0002010BD38B5002000906F
:100940000024002500BF3120FFF7DBFF054600989B
:10095000401C00900098B0F5A06F01D0002DF2D09F
:100960003120FFF7CEFF08B1012400E0002420462B
:1009700038BD01460020A14A106820F0F80040EA86
:10098000C10010607047A04908607047024600200F
:100990009A4B586820F47C1042EA01031843974BA5
:1009A0005860704798490866704701460020934A8E
:1009B000506820F003000843506070478F4840683B
:1009C00000F00C007047014600208C4A506820F06F
:1009D000F00008435060704701460020874A506885
:1009E00020F4E06008435060704701460020834ACD
:1009F000506820F4605040EAC1005060704729B14F
:100A00007E4A527A02437D4B5A7204E07B4A527A04
:100A100082437A4B5A7270477B49D83108607047DD
:100A200001460020754A506820F440400843506059
:100A300070470021714A20321170704A82F82010EC
:100A4000012802D004280AD104E001216B4A203297
:100A5000117005E00521694A2032117000E000BFE5
:100A600000BF70476949086070476449096A0143DB
:100A7000624A11627047654944390860704730B571
:100A800000210022002400235C4D6D6805F00C015C
:100A900021B1042905D0082923D105E05C4D05606A
:100AA00022E05B4D05601FE0544D6D6805F4701247
:100AB000524D6D6805F48034022505EB92421CB955
:100AC000544D554305600BE04C4D6D6805F4003501
:100AD0001DB1504D5543056002E04D4D5543056035
:100AE00002E04B4D056000BF00BF444D6D6805F04E
:100AF000F0010909484D6B5C0568DD4045603F4DDC
:100B00006D6805F4E061090A434D6B5C4568DD40A2
:100B100085603A4D6D6805F46051C90A3E4D6B5CC5
:100B20004568DD40C560354D6D6805F44041890B71
:100B30003A4D6B5CC568B5FBF3F5056130BD29B175
:100B40002E4A526902432D4B5A6104E02B4A5269E6
:100B500082432A4B5A61704729B1284A926902435D
:100B6000264B9A6104E0254A92698243234B9A619D
:100B7000704729B1214AD2690243204BDA6104E06F
:100B80001E4AD26982431D4BDA61704729B11B4A64
:100B9000D2680243194BDA6004E0184AD2688243F3
:100BA000164BDA60704729B1144A12690243134B9D
:100BB0001A6104E0114A12698243104B1A617047AE
:100BC00012494039086070470F49C86470470B49A3
:100BD000C87170470948406A40F080700749486210
:100BE000704701460020054A92680A400AB1012078
:100BF00000E00020704701498872704700100240F1
:100C00000000FFF8FFFFF6FE00004242800442426F
:100C100000127A0000093D0014000020240000208A
:100C200010B50446FE48844208D10121C014FFF7E4
:100C3000ADFF0021E014FFF7A9FFC4E0B4F1804F3D
:100C400008D101210846FFF7AEFF00210120FFF780
:100C5000AAFFB8E0F348844208D101210220FFF73F
:100C6000A2FF00210220FFF79EFFACE0EE48844285
:100C700008D101210420FFF796FF00210420FFF78F
:100C800092FFA0E0E948844208D101210820FFF743
:100C90008AFF00210820FFF786FF94E0E4488442A1
:100CA00008D101211020FFF77EFF00211020FFF75F
:100CB0007AFF88E0DF48844208D101212020FFF735
:100CC00072FF00212020FFF76EFF7CE0DA488442AB
:100CD00008D101214014FFF759FF00216014FFF7EC
:100CE00055FF70E0D548844209D10121C804FFF7BF
:100CF0004DFF00214FF40020FFF748FF63E0D0488C
:100D0000844209D101210805FFF740FF00214FF47B
:100D10008010FFF73BFF56E0CA48844209D1012109
:100D20004805FFF733FF00214FF40010FFF72EFFB7
:100D300049E0C548844208D101214020FFF733FF34
:100D400000214020FFF72FFF3DE0C048844208D13A
:100D500001218020FFF727FF00218020FFF723FFDC
:100D600031E0BB48844208D101218015FFF71BFF09
:100D70000021A015FFF717FF25E0B648844209D1EE
:100D800001210804FFF702FF00214FF48030FFF734
:100D9000FDFE18E0B048844209D101214804FFF764
:100DA000F5FE00214FF40030FFF7F0FE0BE0AB48FA
:100DB000844208D101218804FFF7E8FE00214FF4A6
:100DC0008020FFF7E3FE10BD00220288944B98427A
:100DD0000ED0994B98420BD0B0F1804F08D0914B78
:100DE000984205D0904B984202D0904B984204D143
:100DF0004FF68F731A404B881A438D4B984207D099
:100E00008C4B984204D04FF6FF431A40CB881A43CC
:100E100002808B8883850B880385814B98420BD099
:100E2000854B984208D08B4B984205D08A4B98420C
:100E300002D08A4B984201D10B7A03860123838228
:100E4000704770B5002400220023058C4FF6FE7613
:100E500035400584028C8388048B4FF68F752C40B7
:100E6000B51E2C400D882C43751E2A400D892A433F
:100E70004D882A436A4DA8420BD06F4DA84208D036
:100E8000744DA84205D0744DA84202D0734DA842BB
:100E900013D14FF6F7752A404D892A434FF6FB755B
:100EA0002A408D882A434FF6FF652B404FF6FF55A9
:100EB0002B408D892B43CD892B4383800483CD88A0
:100EC0008586028470BD70B5002400220023058C45
:100ED0004FF6EF7635400584028C8388048B48F604
:100EE000FF752C404FF6FF452C400D884FF6FF76DE
:100EF00006EA05252C434FF6DF752A400D8906EAE0
:100F000005152A434D8806EA05152A43444DA84293
:100F100002D0494DA8421DD14FF67F752A404D8918
:100F20004FF6FF7606EA05152A434FF6BF752A40AD
:100F30008D8806EA05152A434FF6FF352B404FF200
:100F4000FF752B408D8906EA85052B43CD8906EA7E
:100F500085052B4383800483CD880587028470BD7B
:100F600070B5002400220023058C4FF6FF66354043
:100F70000584028C8388848B4FF68F752C404FF646
:100F8000FC752C400D882C434FF6FF552A400D89E7
:100F90004FF6FF7606EA05252A434D8806EA052521
:100FA0002A431F4DA84202D0234DA8421DD14FF223
:100FB000FF752A404D894FF6FF7606EA05252A433C
:100FC0004FF6FF352A408D8806EA05252A434EF65E
:100FD000FF752B404DF6FF752B408D8906EA0515F0
:100FE0002B43CD8906EA05152B4383808483CD8866
:100FF0008587028470BD70B5002200230024058C13
:101000004EF6FF7635400584038C8488828B48F643
:10101000FF752A404FF6FF452A400D8820E000006A
:10102000002C01400004004000080040000C00407B
:10103000001000400014004000340140004C01400A
:10104000005001400054014000180040001C0040C6
:1010500000200040004001400044014000480140A1
:101060004FF6FF7606EA05252A434DF6FF752B401D
:101070000D8906EA05352B434D8806EA05352B43D5
:10108000FA4DA84202D0FA4DA84208D14BF6FF759E
:101090002C408D894FF6FF7606EA85152C43848017
:1010A0008283CD88A0F84050038470BD828B4FF2BC
:1010B000FF331A408283828B4FF6FF7303EA0123CA
:1010C0001A4382837047F0B50C4615460022002172
:1010D0000026078C4EF6FF7C07EA0C070784828BFC
:1010E000018C4FF6FF7707EA043640F6FF473A4097
:1010F0004FF6FF7707EA05273A434FF6FF7707EAEF
:1011000003373A43D94FB8420ED0D94FB8420BD02B
:10111000B0F1804F08D0D74FB84205D0D64FB84273
:1011200002D0D64FB84206D14DF6FF77394046F48B
:101130008057394305E047F6FF57394044F480575C
:10114000394382830184F0BD828B4FF6F3731A40DA
:101150008283828B0A4382837047F0B50C46154622
:10116000002200210026078C4FF6FF6C07EA0C07CF
:101170000784828B018C4FF6FF7707EA04264FF62F
:101180000C773A404FF6FF7707EA03172F433A43AD
:10119000B64FB8420ED0B64FB8420BD0B0F1804F28
:1011A00008D0B44FB84205D0B34FB84202D0B34FC5
:1011B000B84206D14FF6FF57394046F4807739439D
:1011C00005E04FF2FF57394044F48077394382837A
:1011D0000184F0BD028B4FF2FF331A400283028B71
:1011E0004FF6FF7303EA01231A4302837047F0B5F9
:1011F0000C461546002200210026078C4FF6EF7C96
:1012000007EA0C070784028B018C4FF6FF7707EA89
:10121000041640F6FF473A404FF6FF7707EA0337D8
:101220003A434FF6FF7707EA05273A438F4FB84214
:101230000ED08F4FB8420BD0B0F1804F08D08D4FF9
:10124000B84205D08C4FB84202D08C4FB84206D17C
:101250004FF6DF77394046F01007394305E04FF687
:101260005F77394044F01007394302830184F0BDB1
:10127000028B4FF6F3731A400283028B0A430283F8
:101280007047F0B50C46154600220021068C4FF63B
:10129000FE773E400684028B018C4FF60C7632407E
:1012A0007E1C06EA03162E433243704EB0420ED027
:1012B0006F4EB0420BD0B0F1804F08D06D4EB042AF
:1012C00005D06D4EB04202D06C4EB04206D14FF602
:1012D000FD76314044F00106314305E04FF6F576E6
:1012E000314044F00106314302830184F0BD70B502
:1012F00005460C465D4885420ED05D4885420BD0C0
:10130000B5F1804F08D05B48854205D05A488542E8
:1013100002D05A48854200D100E000BF208850B971
:101320002389A28861882846FFF7ABFFE188284619
:10133000FFF79EFF25E0208804280AD12389A28890
:1013400061882846FFF753FFE1882846FFF742FFF0
:1013500017E0208808280AD12389A28861882846B6
:10136000FFF7FBFEE1882846FFF7EEFE09E0238940
:10137000A28861882846FFF7A6FEE1882846FFF785
:1013800095FE70BD2DE9F04105460C46002601276B
:10139000608808B9022600E00026A088012801D153
:1013A000022700E001272088A0B92389A28861884C
:1013B0002846FFF766FFE1882846FFF759FF238993
:1013C0003A4631462846FFF712FFE1882846FFF7E4
:1013D00001FF13E02389A28861882846FFF707FFF1
:1013E000E1882846FFF7F6FE23893A46314628462B
:1013F000FFF747FFE1882846FFF73AFFBDE8F08195
:101400000A884B881A438B881A43CB881A430B8966
:101410001A434B891A438B891A43A0F8442070471A
:101420004FF6FF71818000210180C18041800172EF
:1014300070470021018041808180C180018141810C
:101440008181C1817047002101804180012181801B
:101450000021C1800181704700210180418081808D
:10146000C18001814181818170470000002C0140D1
:10147000003401400004004000080040000C00401F
:1014800021B1028842F00102028004E002884FF696
:10149000FE731A400280704731B1B0F8442042F424
:1014A0000042A0F8442005E0B0F84420C2F30E0248
:1014B000A0F8442070471AB183890B43838102E06E
:1014C00083898B43838170478182704741EA02039D
:1014D000A0F8483070471AB183890B43838102E03A
:1014E00083898B438381704701894FF6F8721140DD
:1014F000018170470A46002101894FF68F73194018
:1015000011430181704730B504460D4629462046F7
:10151000FFF7F0FF208940F00700208130BD2DE962
:10152000F04104460D4616461F46602D06D13B4647
:10153000012231462046FFF75AFE05E03B460122D4
:1015400031462046FFF79DFE29462046FFF7D2FF91
:10155000208940F007002081BDE8F08130B50C46BD
:1015600000210189C9B24FF6FF7505EA032515432D
:1015700025432943018130BD2DE9F04105460E4642
:1015800017469846002443463A4631462846FFF718
:10159000E5FF2C894FF6F870044044F007044FF63D
:1015A0008F70044044F070042C81BDE8F081F0B5E8
:1015B00004460D4616461F463B46324629462046FF
:1015C000FFF7CCFF208940F480402081F0BD0185E9
:1015D000828270470A46002101884FF68F731940B6
:1015E000114301807047F0B50C4615461E46002198
:1015F000002200230189028B038C4FF6F8773940D3
:1016000021434FF6FC473A4040F201173A434FF668
:10161000DD773B404FF6FF7707EA06172F433B4342
:10162000018102830384F0BD0A460021018B4FF63D
:101630008F7319401143018370470A460021018BC3
:1016400048F6FF7319404FF6FF7303EA022319436C
:10165000018370470A460021818B4FF68F73194032
:101660001143818370470A460021818B48F6FF733E
:1016700019404FF6FF7303EA022319438183704731
:1016800021B1028842F08002028004E002884FF615
:101690007F731A400280704721B1828842F00402B1
:1016A000828004E082884FF6FB731A408280704784
:1016B00021B1828842F00802828004E082884FF6DD
:1016C000F7731A408280704721B1828842F001028C
:1016D000828004E082884FF6FE731A408280704751
:1016E0000A460021018B4FF6F7731940114301831D
:1016F00070470A460021018B4FF2FF7319404FF6E5
:10170000FF7303EA02231943018370470A4600214D
:10171000818B4FF6F77319401143818370470A4656
:101720000021818B4FF2FF7319404FF6FF7303EADC
:1017300002231943818370470A460021018B4FF62B
:10174000FB7319401143018370470A460021018B46
:101750004FF6FF3319404FF6FF7303EA0223194394
:10176000018370470A460021818B4FF6FB731940B5
:101770001143818370470A460021818B4FF6FF3366
:1017800019404FF6FF7303EA022319438183704720
:101790000A460021018B4FF67F73194011430183E4
:1017A00070470A460021018BC1F30E014FF6FF730B
:1017B00003EA02231943018370470A460021818B03
:1017C0004FF67F7319401143818370470A46002109
:1017D000818BC1F30E014FF6FF7303EA0223194315
:1017E000818370470A460021018C4FF6FD73194032
:1017F0001143018470470A460021018C4FF6F773AC
:1018000019401143018470470A460021018C4FF6AC
:10181000DF7319404FF6FF7303EA02131943018483
:1018200070470A460021018C4FF67F7319404FF62E
:10183000FF7303EA02131943018470470A4600212B
:10184000018C4FF6FF5319404FF6FF7303EA022352
:101850001943018470470A460021018C4FF2FF733F
:1018600019404FF6FF7303EA0223194301847047BE
:101870000A460021018C4DF6FF7319404FF6FF73A5
:1018800003EA023319430184704730B50023012471
:101890008C40A3B2048C9C430484048C02FA01F5AE
:1018A000ADB22C43048430BD30B5002304248C40F9
:1018B000A3B2048C9C430484048C02FA01F5ADB2FB
:1018C0002C43048430BD70B5034600200024184624
:1018D000183001258D40ACB21D8CA5431D8409B183
:1018E000082909D100EB6100056825F07005056045
:1018F0000568154305600EE00D1FC5F34E0528442D
:10190000056825F4E045056005684FF6FF7606EAB0
:1019100002263543056070BD21B1028842F0020203
:10192000028004E002884FF6FD731A40028070477F
:1019300021B1028842F00402028004E002884FF6DE
:10194000FB731A400280704721B1828842F0800206
:10195000828004E082884FF67F731A40828070474D
:1019600002884FF6F7731A40028002880A43028009
:10197000704782884FF68F731A40828082880A43AC
:101980008280704702894FF6F8731A4002810289FB
:101990000A430281704702894FF67F731A40028121
:1019A00002890A43028170478184704781857047AC
:1019B000818670470187704781877047A0F8401083
:1019C000704702884FF6FF431A40028002880A439C
:1019D000028070470146888E70470146088F704725
:1019E0000146888F70470146B1F8400070470146B4
:1019F000888C70470146088D704702460020138A84
:101A00000B400BB1012000E000207047CA43028266
:101A1000704730B50246002000230024158A05EAED
:101A20000103958905EA010413B10CB1012000E01E
:101A3000002030BDCA4302827047000010B5044642
:101A4000FB48844209D101218803FFF79FF8002158
:101A50004FF48040FFF79AF832E0F648844209D10B
:101A600001214804FFF79FF800214FF40030FFF7F1
:101A70009AF825E0F048844209D101218804FFF753
:101A800092F800214FF48020FFF78DF818E0EB4822
:101A9000844209D10121C804FFF785F800214FF4E1
:101AA0000020FFF780F80BE0E548844208D10121CF
:101AB0000805FFF778F800214FF48010FFF773F85E
:101AC00010BD2DE9F04786B005460E460024A2461B
:101AD00000BFA1460027B08900B100BF2F462C8A65
:101AE0004CF6FF700440F08804432C82AC894EF61B
:101AF000F3100440B08831890843718908430443D6
:101B0000AC81AC8A4FF6FF400440B0890443AC82FC
:101B100001A8FEF7B4FFC648874202D1DDF810A045
:101B200001E0DDF80CA0A88900F4004040B10AEB08
:101B3000CA0000EB0A1031684900B0FBF1F807E079
:101B40000AEBCA0000EB0A1031688900B0FBF1F81B
:101B50006420B8FBF0F004012009642101FB108926
:101B6000A88900F4004040B1322000EBC900B0FB6E
:101B7000F1F000F00700044308E0322000EB091008
:101B80006421B0FBF1F000F00F0004432C8106B09B
:101B9000BDE8F0874FF41651016000218180C180BB
:101BA00001810C21418100218181704710B50246DD
:101BB0000020108A4FF2FF0318400B884C88234303
:101BC0008C882343CC8823431843108210BD002106
:101BD000018041808180C180704721B1828942F4B7
:101BE0000052828104E082894DF6FF731A4082819F
:101BF0007047F0B50346002400260025002040F67B
:101C00006A17B94200D100BF1846C1F3421401F06F
:101C10001F06012707FA06F5012C01D10C3004E05C
:101C2000022C01D1103000E014301AB107682F43A4
:101C3000076002E00768AF430760F0BD1AB1838A0E
:101C40000B43838202E0838A8B4383827047028A3C
:101C50004FF6F0731A400282028A0A4302827047EA
:101C600082894FF2FF731A40828182890A438281FE
:101C7000704721B1828942F00202828104E08289A8
:101C80004FF6FD731A4082817047028A4FF6DF7368
:101C90001A400282028A0A430282704721B1028AF4
:101CA00042F48042028204E0028A4BF6FF731A403B
:101CB00002827047C1F3080282807047014688881B
:101CC000C0F308007047818941F0010181817047AC
:101CD000028BD2B20283028B42EA01220283704756
:101CE000028B02F47F420283028B0A430283704715
:101CF00021B1828A42F02002828204E0828A4FF679
:101D0000DF731A408282704721B1828A42F010024A
:101D1000828204E0828A4FF6EF731A408282704713
:101D200021B1828A42F00802828204E0828A4FF660
:101D3000F7731A408282704721B1828942F40042CF
:101D4000828103E08289C2F30E028281704721B151
:101D5000828A42F40062828204E0828A4FF2FF7338
:101D60001A4082827047828A4FF6FB731A40828241
:101D7000828A0A438282704721B1828A42F002023B
:101D8000828204E0828A4FF6FD731A408282704795
:101D900002460020B1F5007F00D100BF13880B4040
:101DA0000BB1012000E00020704701F40072B2F591
:101DB000007F00D100BFCA430280704770B5024661
:101DC000002400230025002040F66A16B14200D10D
:101DD00000BFC1F3421501F01F03012606FA03F309
:101DE000012D02D19689334006E0022D02D1168AD8
:101DF000334001E0968A33400C12012606FA04F4BF
:101E00001688344013B10CB1012000E0002070BDF1
:101E100010B50022002340F66A14A14200D100BF91
:101E20000A1201249440A3B2DC43048010BD0000D8
:101E3000003801400044004000480040004C004091
:101E40000050004070B5482000F07EF900F0C4F862
:101E500000F08EF84FF4E13000F0C0F800F0ADFA79
:101E600000F074FC002140F60F6000F0CFFA00F0A3
:101E7000F2FE00F08DFD02220021084600F07FFEF8
:101E800003220021102000F07AFE102320A200215E
:101E9000582000F057FE0C231FA20221002000F062
:101EA00051FE0C2320A20321002000F04BFE102342
:101EB00021A20421002000F045FE0C2322A20621CD
:101EC000002000F03FFE0C2323A20721002000F099
:101ED00039FE00F058FB47F230504FF080418884C3
:101EE00000F09EFB47F230501F49088064210846ED
:101EF00000F0EEFA00F00EFB642000F03FF94FF422
:101F0000FA752C4619480580001D048070BD00003C
:101F10006D2F6D696E0000004C656674203A2020BC
:101F2000202052504D00000052696768743A20200A
:101F3000202052504D000000503A202020493A20E5
:101F40002020443A202020005365745F433A20202B
:101F5000202052504D0000005365745F503A2020FD
:101F600020206D2F6D696E00240800403C04004065
:101F700008B501211020FEF7EFFD4FF40050ADF839
:101F8000000010208DF8030003208DF80200694640
:101F90000F48FEF725FB08BD70B504460D480068E4
:101FA000401C0C490860A04210D14FF40051084871
:101FB000FEF7A9FBC0F10100C5B22A464FF400515B
:101FC0000348FEF7BEFB00200249086070BD000018
:101FD00000100140280000207047000010B586B0B6
:101FE0000446012144F20400FEF7B6FD4FF40070F0
:101FF000ADF8140018208DF8170003208DF8160096
:1020000005A94C48FEF7ECFA4FF48060ADF81400D7
:1020100004208DF8170005A94648FEF7E1FA01945F
:102020000020ADF80800ADF80A00ADF80C00ADF8DE
:1020300010000C20ADF80E0001A93F48FFF741FD4C
:10204000012240F225513C48FFF7D3FD01213A48D7
:10205000FFF7C3FD06B010BD70B504460D46E1B2F2
:102060003548FFF727FE00BF80213348FFF790FE79
:102070000028F9D0204670BD10B5044600BF2021CD
:102080002D48FFF785FE0028F9D02B48FFF716FEF4
:1020900010BD70B504460D4640212748FFF785FE68
:1020A00080212548FFF7B4FE13E021782248FFF78E
:1020B00001FE00BF40212048FFF76AFE0128F9D148
:1020C00040211D48FFF771FE80211B48FFF7A0FE4D
:1020D000641C281EA5F10105E7D170BD0022174B35
:1020E0001A60174A1160174A1060704710B540F225
:1020F00025511148FFF762FED8B10F48FFF7DEFD0A
:10210000C4B20F4800680D49096888420CD90D48CF
:10211000006804700B480068401C0A4908600748C2
:102120000068401C0549086040F225510248FFF74D
:102130006FFE10BD00080140003801403000002053
:10214000340000202C00002010B504466FF004007D
:10215000FEF7C7F9E11704EB5171C1F3C701234A38
:1021600011701046007800EB4001C1EBC0104FF633
:10217000FF7101EAC0001E49088010BD01461C4ADB
:1021800012884A434FF0E0235A6100229A610122EB
:102190001A6100BF4FF0E022106900F001021AB18D
:1021A00000F48032002AF5D000224FF0E0231A61BB
:1021B0009A61704701460D4A12784A434FF0E02376
:1021C0005A6100229A6101221A6100BF4FF0E02299
:1021D000106900F001021AB100F48032002AF5D033
:1021E00000224FF0E0231A619A6170473800002006
:1021F0003A000020002001E0411CC8B20A28FBDBA5
:10220000704710B54FF400617F48FEF796FA4FF41F
:1022100080617D48FEF791FAFFF7ECFF4FF4006113
:102220007948FEF78CFAFFF7E5FF4FF480617648B6
:10223000FEF785FAFFF7DEFF10BD10B54FF4006121
:102240007148FEF77CFA4FF480616F48FEF775FA2B
:10225000FFF7D0FF4FF400616B48FEF76EFA10BD38
:1022600070B50446002528E004F0800028B14FF442
:1022700000616548FEF761FA04E04FF400616248CE
:10228000FEF75DFAFFF7B6FF4FF480615E48FEF798
:1022900054FAFFF7AFFF4FF480615B48FEF74FFA47
:1022A000072D04D14FF400615748FEF746FA600647
:1022B000040EFFF79FFF681CC5B2082DD4DB70BD6C
:1022C00010B54FF400615048FEF739FAFFF792FF5E
:1022D0004FF480614C48FEF730FAFFF78BFF4FF464
:1022E00080614948FEF72BFAFFF784FF4FF4006145
:1022F0004548FEF722FA10BD10B54FF40061424880
:10230000FEF71BFAFFF776FF4FF480613E48FEF7B9
:1023100014FAFFF76FFF4FF480613B48FEF70FFAA6
:10232000FFF768FF10BD70B505460024002619E0D0
:102330006006040E4FF480613348FEF7FEF9FFF7A4
:1023400059FF4FF400613048FEF7DDF908B1601C19
:10235000C4B24FF480612C48FEF7F1F9FFF74AFF51
:10236000701CC6B2082EE3DB15B9FFF7C5FF01E00C
:10237000FFF7A6FF204670BD10B54FF4006122485C
:10238000FEF7DBF9FFF736FF4FF480611E48FEF7DA
:10239000D4F9FFF72FFF4FF400611B48FEF7B3F9A4
:1023A00008B1012400E000244FF480611648FEF7D4
:1023B000C6F9FFF71FFF204610BD08B50121082010
:1023C000FEF7CAFB4FF44060ADF8000003208DF823
:1023D000020014208DF8030069460B48FEF700F94F
:1023E000FFF72BFF08BD70B50446FFF7E6FFFFF7C8
:1023F00008FF2046FFF734FFFFF7BEFF0546FFF753
:102400001CFF284670BD0000000C014030B589B0AB
:1024100005460C4601210220FEF7ABFB681E80B288
:10242000ADF80800A0B2ADF804000020ADF80A0035
:10243000ADF8060001A9C048FEF7C6FC0121BE4860
:10244000FFF7E4FA01221146BB48FFF734F80121F7
:102450000820FEF781FB0320ADF8100018208DF84E
:10246000130003208DF8120004A9B448FEF7B8F851
:102470006020ADF814000120ADF816000020ADF882
:102480001A00ADF81C0005A9AB48FEF769FD08214C
:10249000A948FFF7D3F96020ADF814000120ADF88A
:1024A00016000020ADF81A00ADF81C0005A9A248DE
:1024B000FEF7A1FD0821A048FFF7DAF901219E48A7
:1024C000FFF7DEF801219C48FEF7DAFF09B030BDC6
:1024D0007FB505460C466020ADF800000120ADF840
:1024E0000200ADF8065069469348FEF739FD082111
:1024F0009148FFF7A3F9ADF8064069468E48FEF70C
:102500007AFD08218C48FFF7B3F901218A48FFF7CB
:10251000B7F87FBD1FB501211020FEF72AFB42F25C
:102520000F70ADF8080040F2CF20ADF80400002095
:10253000ADF80A00ADF806008DF80C0001A980483E
:10254000FEF742FC01217E48FFF760FA01221146A6
:102550007B48FEF7B0FF4FF44070FDF773FF362065
:102560008DF8000005208DF8010000208DF8020094
:1025700001208DF803006846FDF769FF01217048CE
:10258000FEF77EFF1FBD00B587B001210846FEF7AC
:10259000F0FA01210420FEF7DFFA0320ADF8000075
:1025A00004208DF8030069466648FEF719F804A870
:1025B000FEF736FF0020ADF810004EF66020ADF8B3
:1025C00014000020ADF81600ADF8120004A94FF079
:1025D0008040FEF7F9FB00231A4603214FF08040AC
:1025E000FFF701F801A8FEF72EFF0A20ADF80C0056
:1025F00001A94007FEF77BFE01218807FFF706FAD5
:10260000012211469007FEF756FF00214FF080404F
:10261000FFF7CAF901218807FEF732FF07B000BDB6
:1026200000B587B001210420FEF7A3FA012108209C
:10263000FEF792FAC020ADF8000004208DF80300E8
:1026400069463E48FDF7CCFF04A8FEF7E9FE0020EE
:10265000ADF810004EF66020ADF814000020ADF883
:102660001600ADF8120004A93748FEF7ADFB0023B1
:102670001A4603213448FEF7B6FF01A8FEF7E3FE31
:102680000A20ADF80C0001A92F48FEF730FE012109
:102690002D48FFF7BBF9012211462B48FEF70BFF2F
:1026A00000212948FFF780F901212748FEF7E8FEBD
:1026B00007B000BD0146022904D003290CD004292B
:1026C0001ED113E04FF08042928C10B247F230528C
:1026D0004FF080439A8415E0174A2432128810B2D2
:1026E00047F23052144B24331A800BE0164A24323E
:1026F000128810B247F23052134B24331A8001E093
:10270000002000BF00BF70470F48103000880E48FF
:102710001030008820F001000B491031088070470C
:102720004FF08040008A4FF08040008A20F0010086
:102730004FF080410882704700040040000C0140C7
:1027400000100040000801400008004008B50121C9
:102750000820FEF701FA4FF47040ADF80000102099
:102760008DF8030003208DF8020069463748FDF715
:1027700037FF08BD10B504464CB94FF480513348BB
:10278000FDF7DBFF4FF400513048FDF7D8FF012C77
:1027900007D161032D48FDF7D0FF21032B48FDF73A
:1027A000CEFF022C07D1E1022848FDF7C8FF210324
:1027B0002648FDF7C4FF10BD10B504464CB94FF4D0
:1027C00000412248FDF7B9FF4FF480411F48FDF753
:1027D000B6FF012C07D1A1031C48FDF7AEFFE103B2
:1027E0001A48FDF7ACFF022C07D161031748FDF72B
:1027F000A6FFA1031548FDF7A2FF10BD10B50020EC
:10280000FFF7B8FF0020FFF7D7FF10BD10B501207C
:10281000FFF7B0FF0120FFF7CFFF10BD10B501207B
:10282000FFF7A8FF0020FFF7C7FF10BD10B500207D
:10283000FFF7A0FF0120FFF7BFFF10BD10B502207A
:10284000FFF798FF0220FFF7B7FF10BD000C014013
:1028500010B50446FFF7D5FC7820FFF701FDFFF720
:102860008BFD0020FFF7FCFCFFF786FD2046FFF7FD
:10287000F7FCFFF781FDFFF7E0FC10BD10B5044643
:10288000FFF7BFFC7820FFF7EBFCFFF775FD40205A
:10289000FFF7E6FCFFF770FD2046FFF7E1FCFFF7CE
:1028A0006BFDFFF7CAFC10BD70B504460D461DB1A7
:1028B000E0B2FFF7E3FF02E0E0B2FFF7C9FF70BD4F
:1028C00070B50646002418E004F1B0000021FFF7BF
:1028D000EBFF00210846FFF7E7FF00211020FFF77C
:1028E000E3FF002505E001213046FFF7DDFF681C0E
:1028F000C5B2802DF7DB601CC4B2082CE4DB70BDD0
:1029000006E041F6650100E0491E0029FCD1401EA9
:102910000028F6D17047014605E0002001E0421C86
:10292000D0B27B28FBDB0A1EA1F10101F5D1704773
:1029300070B504460D4605F1B0000021FFF7B4FF65
:10294000102141EA14100021FFF7AEFF04F00F0040
:102950000021FFF7A9FF70BD10B500218D20FFF702
:10296000A3FF00211420FFF79FFF0021AF20FFF7F6
:102970009BFF10BD10B500218D20FFF795FF0021B2
:102980001020FFF791FF0021AE20FFF78DFF10BD53
:1029900070B5002418E004F1B0000021FFF784FFB7
:1029A00000210846FFF780FF00211020FFF77CFF81
:1029B000002505E001210020FFF776FF681CC5B265
:1029C000802DF7DB601CC4B2082CE4DB70BD70B551
:1029D000002418E004F1B0000021FFF765FF00219A
:1029E0000846FFF761FF00211020FFF75DFF00257B
:1029F00005E001210846FFF757FF681CC5B2802D8E
:102A0000F7DB601CC4B2082CE4DB70BD2DE9F04795
:102A100007460E469046994600250024A8F120005E
:102A2000C5B27F2F02DD0027B01CC6B2B9F1100F6E
:102A300024D131463846FFF77BFF002408E004EB41
:102A40000511BF4A505C0121FFF72EFF601CC4B284
:102A5000082CF4DB701CC1B23846FFF769FF002474
:102A600009E004EB05110831B54A505C0121FFF77C
:102A70001BFF601CC4B2082CF3DB12E03146384661
:102A8000FFF756FF00240AE005EB4501AD4A02EBD3
:102A90004101085D0121FFF707FF601CC4B2062C4D
:102AA000F2DBBDE8F08710B50246012000E050439C
:102AB0000B1EA1F10104E1B2F9D110BD2DE9FF5FB8
:102AC000074691461E460E9D4FF0000A002435E051
:102AD000301B401EC1B20A20FFF7E5FFB9FBF0F042
:102AE0000A21B0FBF1F201FB1208BAF1000F14D178
:102AF000701EA04211DDB8F1000F0CD1AB4605EB02
:102B0000DB71491001FB0471C8B22B4620220199E8
:102B1000FFF77CFF10E04FF0010AAB4605EBDB71DD
:102B2000491001FB0471C8B208F13001CAB22B464A
:102B30000199FFF76BFF00BF601CC4B2B442C7DB52
:102B4000BDE8FF9F2DE9F04104460F461546984623
:102B500000260FE0AA5D434639462046FFF756FFA0
:102B600004F10800C4B2782C02DD0024B81CC7B2FE
:102B7000701CC6B2A85D0028ECD1BDE8F0812DE93B
:102B8000F04180460E461546002731464046FFF785
:102B9000CFFE00240AE06C4A02EB8511085D01219A
:102BA000FFF782FE781CC7B2601CC4B2102CF2DBA7
:102BB000701CC1B24046FFF7BBFE00240CE0690068
:102BC000491C614A02EB4111085D0121FFF76CFECF
:102BD000781CC7B2601CC4B2102CF0DBBDE8F081D9
:102BE0002DE9F05F06460F4690461C46DDF828A00A
:102BF0004FF0000BE11704EB5171C910A4EBC101B8
:102C000031B92046E11704EB5171C1F3C70506E065
:102C10002046E11704EB5171C910491CCDB23D4665
:102C200015E029463046FFF783FEB1460BE05946D2
:102C30000BF1010B1AF801000121FFF735FE09F134
:102C4000010000F0FF09C145F1DB681CC5B2A542D7
:102C5000E7DBBDE8F09F10B5FFF7AFFB4FF448701E
:102C6000FFF78CFA0021AE20FFF71EFE0021084678
:102C7000FFF71AFE00211020FFF716FE002140206A
:102C8000FFF712FE0021B020FFF70EFE0021812089
:102C9000FFF70AFE0021FF20FFF706FE0021A1201A
:102CA000FFF702FE0021A620FFF7FEFD0021A8206D
:102CB000FFF7FAFD00213F20FFF7F6FD0021C820B5
:102CC000FFF7F2FD0021D320FFF7EEFD00210846BB
:102CD000FFF7EAFD0021D520FFF7E6FD0021802067
:102CE000FFF7E2FD0021D820FFF7DEFD00210520DF
:102CF000FFF7DAFD0021D920FFF7D6FD0021F120F2
:102D0000FFF7D2FD0021DA20FFF7CEFD00211220CF
:102D1000FFF7CAFD0021DB20FFF7C6FD00213020B0
:102D2000FFF7C2FD00218D20FFF7BEFD002114201A
:102D3000FFF7BAFD0021AF20FFF7B6FD10BD000080
:102D4000C24C00089A4A00083C0000202DE9FE43CE
:102D500055480468204601F09BFC064632460B4667
:102D600052A102A800F000FB102302AA0421184679
:102D7000FFF7E8FE4F480568284601F089FC064643
:102D800032460B4649A101A800F0EEFA102301AA31
:102D900004213820FFF7D6FE4748D0F8008040468F
:102DA00001F076FC064632460B4640A1684600F02C
:102DB000DBFA10236A4604216820FFF7C3FEBDE852
:102DC000FE832DE9FC5F04460D462E1B3B48006840
:102DD00001F008FD834638480168584601F01AFDA5
:102DE00081463748006801F0FDFC009031480168D9
:102DF000009801F00FFD8346304601F0F3FC00908F
:102E000029480168009801F005FD5946019001F03C
:102E1000CDFD8246494601F067FC804601F0C6FCC4
:102E20000746274800682549086025480660384657
:102E3000BDE8FC9F2DE9FC5F04460D462E1B214892
:102E4000006801F0CFFC83461B480168584601F03A
:102E5000E1FC81461C48006801F0C4FC0090154864
:102E60000168009801F0D6FC8346304601F0BAFCB8
:102E700000900D480168009801F0CCFC5946019083
:102E800001F094FD8246494601F02EFC804601F097
:102E90008DFC07460C4800680A4908600A4806602D
:102EA0003846BDE8FC9F00003C02002025312E3151
:102EB0006600000040020020440200204C02002076
:102EC0004802002054020020500200202DE9F84F53
:102ED00001217D48FEF791FD00287DD001217A482F
:102EE000FEF7A8FD0520FFF757F80220FFF7E2FBE9
:102EF000A0F5EA403038754908600420FFF7DAFB96
:102F0000A0F5EA40303872490860084600686F4909
:102F1000096800EB010A0AEBDA7040104FF41671F1
:102F200048434FF41C6190FBF1FB584601F09BFABB
:102F30008046684A684B01F0ADFA0646674A684B1E
:102F400001F0A8FA044601F05DFA664908600846F7
:102F5000006801F09DFB044622460B4662A16448CE
:102F600000F002FA1023624A00213020FFF7EAFD48
:102F700056480068002804DA544800684042534923
:102F8000086053480068002804DA5148006840424D
:102F90004F490860574800684FF41C6148434FF49C
:102FA000167190FBF1F4214648480068FFF709FFCD
:102FB000514908604F4800684FF41C6148434FF482
:102FC000167190FBF1F4214641480068FFF732FF8B
:102FD0004A490860484800E073E0006810F1030FB8
:102FE00003DB45480068032806DD45480068424980
:102FF00009680844424908604048006810F1030F1E
:1030000003DB3E480068032806DD3E4800683B4974
:10301000096808443B4908603948006840F6AC51EB
:10302000884203DD40F6B83035490860354800680D
:1030300040F6AC51884203DD40F6B83031490860B3
:1030400040F2DC502E4908602E4908602C48008868
:103050002D4908802B480088091D0880FFF776FE5F
:103060001A4800684FF4167148434FF41C6190FBF6
:10307000F1F0264908600C20032300900846022145
:1030800002683820FFF71AFD114800684FF41671E6
:1030900048434FF41C6190FBF1F01D4908600C207F
:1030A000032300900846194602683820FFF706FD02
:1030B0000C20032300900F48062102683020FFF700
:1030C000FDFCBDE8F88F0000001000405802002011
:1030D0005C020020A4703D0AD7A3B03F6F1283C0EA
:1030E000CA2109407C02002025322E3266000000F1
:1030F0008902002070020020680200206C0200207B
:1031000060020020640200203C04004074020020A1
:103110007802002010B586B0044601210420FDF796
:103120001BFD01214804FDF724FD0420ADF8140027
:1031300018208DF8170003208DF8160005A94648C1
:10314000FDF74EFA0820ADF8140004208DF81700A2
:1031500005A94148FDF744FA01940020ADF80800A4
:10316000ADF80A00ADF80C00ADF810000C20ADF879
:103170000E0001A93948FEF7A4FC4FF4E060FDF70A
:1031800061F926208DF8000000208DF801008DF8EF
:10319000020001208DF803006846FDF758F901226E
:1031A00040F225512D48FEF724FD01212B48FEF762
:1031B00014FD06B010BD70B504460D4640212748E9
:1031C000FEF7F3FD80212548FEF722FE13E021786B
:1031D0002248FEF76FFD00BF40212048FEF7D8FDD2
:1031E0000128F9D140211D48FEF7DFFD80211B4851
:1031F000FEF70EFE641C281EA5F10105E7D170BD87
:103200000022174B1A60174A1160174A1060704766
:1032100010B540F225511148FEF7D0FDD8B10F4846
:10322000FEF74CFDC4B20F4800680D49096888429A
:103230000CD90D48006804700B480068401C0A490E
:10324000086007480068401C0549086040F22551A5
:103250000248FEF7DDFD10BD0008014000440040BB
:10326000940200209802002090020020FEF7EAFD60
:103270004FF41650FFF74EFFFFF7E0FA64E014201A
:10328000FEF77CFF06213148FFF7BAFF06212F48E1
:10329000FFF791FF2D48C078B12806D12B4800795F
:1032A000B52802D100202949C8702848C078B32821
:1032B00006D126480079B72802D100202349C870DA
:1032C0002248C078B22805D120480079B62801D11B
:1032D000FFF794FA1D48C078B4280ED11B48007936
:1032E000B8280AD1FFF79AFA4FF4FA70FEF746FFB2
:1032F000FFF784FA00201549C8701448C078B52833
:1033000005D112480079B92801D1FFF797FA0F4883
:10331000C078B6280ED10D480079BA280AD1FFF737
:1033200085FA4FF4FA70FEF729FFFFF767FA0020DD
:103330000649C8700548C078B82805D10348007907
:10334000BC2801D1FFF762FA99E700009C02002037
:10335000704700BFFEE700BFFEE700BFFEE700BF0B
:10336000FEE77047704770470FB41CB5074B06AABD
:103370007B4469460090059800F0CDFA002069462C
:1033800000F0DCFA1CBC5DF814FB0000C90500006D
:1033900070B5044685690068C10601D5302600E095
:1033A0002026C00707D070BDD4E9012130469047E0
:1033B000206A401C20626D1EF6D570BD70B50446B3
:1033C00085690078C00707D170BDD4E901212020AC
:1033D0009047206A401C20626D1EF6D570BD2DE915
:1033E000F0474FF0000A89460446C0F820A0204666
:1033F000E1688847002876D0252806D0D4E9012145
:103400009047206A401C2062F1E7E16820460025D1
:103410008847C4F81CA006460027C4F818A02A2E26
:1034200009D0304600F0D0FF38B304EB8708303EB7
:10343000C8F8186019E059F8041B204604EB87020D
:103440009161E1688847012F064618D1E06900289C
:1034500020DA25F020051DE0D8F8180000EB8000E8
:1034600006EB40003038C8F818002046E16888476D
:10347000064600F0A9FF0028EED1012F0AD02E2E1B
:1034800008D12046E16888477F1C0646022F45F098
:103490002005C4DBA069002803DA404245F001059D
:1034A000A061E80701D025F01005B6B1A6F14100F2
:1034B000192802D8203645F400654A463146204690
:1034C00025604D46FCF78EFE58B1012806D0ED1D53
:1034D00025F0070000F1080989E704E005F1040977
:1034E00085E730468AE7206ABDE8F0877047704775
:1034F000704770472DE9FF4F0C461E464FF0FF37CF
:103500008BB0D2E90001DDF860800A908A46C1F3F1
:103510000A5505B93D46002108464FF00000BAF1B2
:10352000000F00F4400005DA00EB80004FF440018A
:1035300001EA50004FEA9059B9F1010F00DDB94698
:103540000A9850EA4A000ED044F61050A5F2FF3512
:1035500045432F14B8F1000F1ED07542291E1EDD01
:10356000C9F100021CE0B8F1010F4FF0000001D0DA
:10357000302103E0F24305E02154401CB042FBDB64
:1035800030460022002121540B99C1F80880C1E97E
:1035900000200FB0BDE8F08FBD1B6D1CDEE74A4672
:1035A00000DA694206A800F059FA06AB93E8070072
:1035B00003AB83E8070050460A9900F036FB8DE81C
:1035C0000700A0F500501F3800900398002D09DD7A
:1035D00042F21F014A46084403A90390684600F0DE
:1035E00095FD08E0A0F500504A461F3803A9039056
:1035F000684600F09FFD8DE807000004000C03D032
:103600004FF0FF30410800E01046B8F1000F03D042
:103610000022009215461EE0751E05D400F098F9B0
:10362000303262556D1EF9D5B3460122084302D0EF
:1036300000227F1C04E02078302801D100227F1E68
:10364000002A099786D01DE0112D07DA00F080F9D5
:10365000303262556D1C50EA0102F5D1084302D0A8
:103660000098C8B10EE00021681E05E0235C625C92
:1036700063542254401E491C8142F7DBAB46A81B11
:10368000401E0990002004F80B000B98099AC0F81E
:103690000880C0E9002B7CE711264FF0000859E7AD
:1036A0002DE9F04F88460446D21D22F0070191B063
:1036B000D1E90001CDE90A0100F072FE02460B9843
:1036C000C00F01D02D2007E02068810701D52B20F5
:1036D00002E0202101EAC000032A099001D0072A54
:1036E00005DB03464146204600F078F90BE12078DF
:1036F000800601D5E06900E00620B8F1650F81463B
:1037000006D0B8F1660F18D0B8F1670F70D131E06C
:103710000020B9F1110F009001DB112301E009F144
:1037200001030AAA01A90CA8FFF7E4FEDDE90C7069
:10373000002609F10105834647E001204B46009031
:103740004FF000470AAA01A90CA8FFF7D3FEDDE954
:103750000DB00C995D46002610B909F101000D1855
:10376000B9EB050003D4C0F1FF3609F10105A5EB63
:1037700009002BE0B9F1010F01DA4FF00109002037
:10378000B9F1110F0090484601DD112300E0034616
:103790000AAA01A90CA8FFF7ADFEDDE90C704D46A1
:1037A00000268346207800070AD4AB4500DA5D4640
:1037B00001A8012D04DD411911F8011C302907D0A1
:1037C0004F4502DA17F1040F04DA012082460FE0B8
:1037D0006D1EEEE7002F02DCED1B3E4403E0781C7B
:1037E000A84200DD7D1CB81B00F1010A4FF0004724
:1037F0002078000703D4AA4501DB4FF0FF3A0021EF
:10380000B7F1004F0DF143088DF8431024D002208A
:103810002B23002F01DA7F422D230A21021EA0F163
:10382000010000DC5FB197FBF1FC97FBF1F201FBBB
:103830001C7C17460CF1300C08F801CDEEE7A8F11E
:10384000010003702188090501D5452100E06521AB
:10385000A0F1010800F8011C09980FA9A1EB0807C5
:10386000FF1D00B10120411901EBEA70A169384444
:10387000081A401EA0612078C00602D42046FFF737
:1038800087FD099828B1D4E901219047206A401C9E
:1038900020622078C00622D52046FFF779FD1EE081
:1038A000002E04DBB34502DD01A8805D00E030207E
:1038B000D4E901219047206A401C2062761CAAF1BD
:1038C00001005FEA000A0AD100F03EF8C068016812
:1038D000405CD4E901219047206A401C2062281EE8
:1038E000A5F10105DCDC07E0D4E9012118F8010BA2
:1038F0009047206A401C2062381EA7F10107F3DCC4
:103900002046FFF75BFD032011B043E601694A1C26
:1039100002610878704700B58FB0CDE90131002110
:10392000059105497944CDE9031011466846FFF732
:1039300056FD0FB000BD0000E5FFFFFF0A6802F86A
:10394000010B0A607047000000487047FC0200202D
:1039500030B5B0F10A024FEA900E71F100034EEA61
:10396000817EB0EB0E0061EB91014FEA101E4EEA32
:10397000017E10EB0E0041EB11114FEA102E4EEAC2
:10398000016E10EB0E0041EB11214FEA104E4EEA92
:10399000014E10EB0E0041EB1141401841F10001C6
:1039A0004FEAD00040EA41704FEAD10110EB8005A8
:1039B0004FEA810444EA907444EB01046D1944EB2E
:1039C0000404521BA3414FF0000348BF0A3200D544
:1039D00030BD401C41F1000130BD00002DE9F04137
:1039E0001F46044603260168072A01F4006004DB31
:1039F00008B116A505E016A503E008B115A500E07D
:103A000015A521F010002060A069C01EA0610FB1B3
:103A1000401EA0612046FFF7BBFC4FB1D4E9012155
:103A200038469047206A401C2062C01C206206E095
:103A3000206AFAE7D4E9012115F8010B9047761EB8
:103A4000F8D22046FFF7BAFCBDE8F0814E414E00A7
:103A50006E616E00494E4600696E66002DE9F047C2
:103A6000814616468AB0334878440DC88DE80D006B
:103A700030487844801C03AC0DC884E80D0041F642
:103A80009B300844372190FBF1F290FBF1F5A5F152
:103A9000800501FB12041B3C02D56442012000E0BA
:103AA0000020DFF890A080460027FA44AAF1BE0A61
:103AB0000DE0E00709D03246684607EB47010AEB04
:103AC000810100F037FB8DE8070064107F1C002C9B
:103AD000EFD1184F7F44AC3F18E0E80714D007EB54
:103AE00004100DF1180A90E80E008AE80E00C06874
:103AF000F04201D198190890324606A903A800F0B7
:103B000019FB03AB83E807006D10641C002DE4D1A2
:103B100032466946B8F1000F03A802D000F0F6FA69
:103B200001E000F007FBC9E90001C9F808200AB06C
:103B3000BDE8F087C418000000487047DC02002090
:103B40007546FFF7F9FFAE4605006946534620F07B
:103B50000700854618B020B5FCF772FBBDE8204091
:103B60004FF000064FF000074FF000084FF0000B39
:103B700021F00701AC46ACE8C009ACE8C009ACE8EC
:103B8000C009ACE8C0098D46704710B50446AFF3D4
:103B900000802046BDE81040FCF73EBB4FF0013CE2
:103BA00050F8042B51F8043B9A4221D1A2EB0C03AC
:103BB000934313EACC1317D150F8042B51F8043B6C
:103BC0009A4215D1A2EB0C03934313EACC130BD109
:103BD00050F8042B51F8043B9A4209D1A2EB0C0394
:103BE000934313EACC13DBD04FF00000704700BFC3
:103BF000D01A01BAB1FA81F101F0180122FA01F0EC
:103C0000CB40C1F12001DBB2C0B2C01A2CFA01F3E3
:103C1000D11A914311EAC311E6D170470149182026
:103C2000ABBEFEE72600020070475FEA400C08BF0B
:103C300091F0000F4FEA8C234FEAC12243EA515121
:103C40004FEA1C5018BF00F5F0404FEA300018BF93
:103C500041F000415FEA6C5C00F02980BCF1FF3F5D
:103C600008BF40F080407047130C06BF12044FF0AD
:103C7000100C4FF0000C130E04BF12020CF1080CD4
:103C8000130F04BF12010CF1040C930F04BF920038
:103C90000CF1020CD30F04BF52000CF1010C1146C1
:103CA0004FF00002A0F11F00A0EB0C00704711F0D4
:103CB000004F08BF704731F000413FF4D5AF0B0C07
:103CC00006BF09044FF0100C4FF0000C0B0E04BFA0
:103CD00009020CF1080C0B0F04BF09010CF1040CD4
:103CE0008B0F04BF89000CF1020CCB0F04BF4900FD
:103CF0000CF1010CCCF12003A0EB0C0022FA03F331
:103D000002FA0CF241EA030100F10100704720F0D1
:103D10007F4C80EA030023F07F47ACEB070303F5F9
:103D20007C5300F0004003F1FF032DE980494FEA86
:103D3000154B09B44FEA144325EA0B4E24EA034815
:103D40000FF2042606EB132749083E785FEA320299
:103D500003FB0667C7F5000707FB06F64FEA543773
:103D60004FEAD64606F1020607FB066CCCF1005C72
:103D70004FEA1C472CEA074C07FB06F40CFB06F540
:103D800004EB15464FEA961634BF00204FF0004072
:103D90004FEAD13706FB07FC4FEA1C4C0CFB0BF734
:103DA000D21B03FB0CF761EB07010CFB0EF7B0EB2A
:103DB000074072EB17420CFB08F734BFA2EB074237
:103DC000B2EB074261EB17414FEA0C444FEA91070F
:103DD00006FB07FC4FEA1C4C0CFB0BF7B0EBC74093
:103DE00072EB573203FB0CF734BFA2EBC742B2EBC6
:103DF000C74261EB57310CFB0EF7B0EBC70072EB1B
:103E000057720CFB08F734BFA2EBC702B2EBC70234
:103E100061EB5771039F4FEA816141EA921104EB14
:103E2000CC044FEAD1374FEA826206FB07FC42EA34
:103E300090124FEA80604FEA1C4C0CFB0BF7D21B30
:103E400003FB0CF761EB07010CFB0EF7B0EB07402F
:103E500072EB17420CFB08F734BFA2EB0742B2EB40
:103E6000074261EB17414FEA8C554FEA910704EB8B
:103E70009C2406FB07FC4FEA1C4C0CFB0BF7B0EB39
:103E8000C74072EB573203FB0CF734BFA2EBC742BB
:103E9000B2EBC74261EB57310CFB0EF7B0EBC7003A
:103EA00072EB57720CFB08F734BFA2EBC702B2EB00
:103EB000C70261EB577115EB4C254FEA816141EA6E
:103EC00092114FEA82624FEAD13742EA901206FB22
:103ED00007FC44F100044FEA80604FEA1C4C0CFBE5
:103EE0000BF7D21B03FB0CF761EB07010CFB0EF782
:103EF000B0EB074072EB17420CFB08F734BFA2EBA4
:103F00000742B2EB074261EB174115EB1C154FEA74
:103F1000813141EA92414FEA823242EA90424FEACD
:103F200080304FEA0C7644F1000448EA03434EEA3D
:103F30000B484FF0000EB2EB080C71EB030724BFE7
:103F4000624639464EEB0E0E4FF0000B0018524100
:103F500049414BEB0B0BB2EB080C71EB03077BF108
:103F6000000B24BF624639464EEB0E0E4FF0000B9D
:103F70000018524149414BEB0B0BB2EB080C71EBB3
:103F800003077BF1000B24BF624639464EEB0E0E51
:103F900051EA020718BF46F0010616EB0E7655F1FE
:103FA000000254F1000103D5BDE88901BDE8008895
:103FB000BDE88901BDE80048B619524141EB010155
:103FC000A3F10103704780807F7E7D7C7B7A7978C6
:103FD000777676757473727171706F6E6E6D6C6CCE
:103FE0006B6A6A6968686766666564646363626170
:103FF0006160605F5F5E5E5D5D5C5C5B5B5A5A59F1
:10400000595858575756565555555454535352525C
:104010005251515050504F4F4F4E4E4D4D4D4C4CB4
:104020004C4B4B4B4A4A4A494949484848474747FD
:10403000474646464545454444444443434343423A
:10404000424242414141002B26D4770021D01CB589
:104050004FEA370703B44FF010004FF010014FF054
:1040600000000FBCBDE810400BF1010BBBF1010FCC
:1040700008BF5FEA170722BF12F1010211F1010127
:104080004FF0004143F1000300F0004043EA00001C
:104090007047F9D35708DAE746EA064613F1400FAE
:1040A0004FEA16461FDD13F1200FDFBF16430A4605
:1040B000002120335B42C8D0C3F1200746EA064600
:1040C00002FA07F74FEA164646EA0706C3F1200749
:1040D00022FA03F201FA07F721FA03F14FF0000385
:1040E00042EA0702B1E746EA020646EA06464FEA16
:1040F000164646EA0106BCBF46EA0646360C4FF0B5
:1041000000034FF000024FF000019EE72DE9C04888
:10411000934630B491E8380007C831EA400C48BFF4
:1041200034EA430C03D5FFF7F2FDFFF78CFFF0BC38
:10413000BDE800882DE9C048934630B491E83800C6
:1041400007C810F0804F08BF13F0804F03D100F074
:1041500005F8FFF778FFF0BCBDE8008820F07F4746
:1041600080EA030023F07F4C07EB0C03A3F57C539C
:1041700000F00040A3F1FE0392F0000F00F0B380C6
:1041800095F0000F00F077802DE901494FEA1140CA
:104190004FEA144621EA004800FB06FC24EA0647E1
:1041A00008FB06F607FB08F800FB07F718EB0648C4
:1041B0004CEB164C4FEA124B18EB07484FEA1546EA
:1041C0004CEB174022EA0B4E0BFB06FC25EA064798
:1041D0000EFB06F607FB0EFE0BFB07F71EEB064E6B
:1041E0004CEB164C4FF000061EEB074E4CEB174BFA
:1041F00018EB0B0840F1000018EB0E0B58EB000811
:1042000040F100008F1A4FF000013CBFC943661B0C
:1042100014BFB5EB040C00213CBFC943F61B4FEAA9
:1042200017444EEA8E0E27EA04454FEA1C4704FB6A
:1042300007622CEA074C05FB07F70CFB05F604FBAD
:104240000CFC16EB074642EB174216EB0C4642EB12
:104250001C421BEB060658EB0202414146EA9E0651
:1042600001D5BDE80189B619524141EB0101A3F125
:104270000103BDE801894FEA14454FEA114724EADA
:10428000054621EA074C05FB07F406FB07F70CFB84
:1042900006F105FB0CFC11EB074144EB17444FEA18
:1042A000124711EB0C4144EB1C4422EA074C05FB7E
:1042B00007F206FB07F70CFB06F605FB0CFC16EBFA
:1042C000074642EB174216EB0C4642EB1C456A18B8
:1042D00054F1000148BF7047B619524141EB01014A
:1042E000A3F10103704795F0000F37D04FEA114258
:1042F0004FEA144721EA024624EA074C02FB07F181
:1043000006FB07F70CFB06F402FB0CFC14EB07445E
:1043100041EB17414FEA154714EB0C4441EB1C41AC
:1043200025EA074C02FB07F506FB07F70CFB06F630
:1043300002FB0CFC16EB074645EB174516EB0C464B
:1043400045EB1C42121951F1000148BF7047B619E4
:10435000524141EB0101A3F1010370474FEA1445BB
:104360004FEA114724EA054621EA074C05FB07F10D
:1043700006FB07F70CFB06F24FF0000605FB0CFCF2
:1043800012EB074241EB174112EB0C4251EB1C417F
:1043900048BF7047921841EB0101A3F10103704738
:1043A000490050EAC12018BF04204A0D18BF40F050
:1043B000010040F2FF72B2EB515F08BF40F0020013
:1043C000012808BF0520704730380A2801D2012093
:1043D000704700207047000010B500290AD0087807
:1043E000002807D005487844FFF7D8FB002801D003
:1043F000002010BD0248784410BD0000820F00006C
:104400007A0F000021F00042A2F16052B2F5801F45
:1044100001F0004328BFD2F17F6C0BD95FEA001C8A
:1044200043EAC20242EB507018BF704728BF20F029
:1044300001007047B2F5801FBCBF184670474FEAB5
:10444000410C1CF5001F02D2084600F0AABA70B554
:1044500000F0CAF800000089FFF7F6BF4FF00040F7
:10446000A0F58000704710F0004248BF4042B0FA0B
:1044700080F310FA03F10AD0C3F11D0303F5806342
:104480004FEA415002EB035202EBD12170474FF04B
:1044900000007047DFF848C170B51CEA111E1EBF4E
:1044A0001CEA13159EEA0C0F95EA0C0F00F06F80C2
:1044B00081EA030423EA4C134EEAD47E21EA4C112C
:1044C00041F4801143F48013AE44A1FB024CA0FBE5
:1044D0000365AEF17F7E361955EB0C05A1FB034C4D
:1044E0004CF10003A0FB021C16EB0C06654153F1D6
:1044F0000003094218BF46F0010613F4007F0BD1F8
:104500004FEA03314FEA0530340341EA155140EADE
:1045100016506FF003020AE04FEAC3214FEAC520AC
:10452000F40241EA555140EA56506FF0020202EBA4
:104530002E4201EB025585EACE710AD05FEA440CA7
:1045400018BF24F0004450F1000041F1000120EABE
:10455000D47040F2FE7C624500D270BDA84214BF08
:104560004FF080444FF04044002E08BF0024BEF1BD
:10457000806FA8BFA1F1C041BDE8704080F2828089
:104580004FF0000001F1C04101F0004170479EEA88
:104590000C0F0CEA131518BF95EA0C0F06D04FF05C
:1045A000000081EA030E0EF0004170BD00F01CF81F
:1045B0008900013E00F007B800F009B84FEA430C4B
:1045C0005FEA5C5C08D081EA030100F05BB84FEA67
:1045D000410C5FEA5C5CF6D14FF000000149704786
:1045E0000000FF070000F87F0EF1020E2EF0030E10
:1045F0005EF8046B364205D4012A43EB030515F53A
:10460000001F12D8012841EB010C1CF5001F0CD82B
:104610000ED14FEAD17C15F5001F0CEB4C0C0CF1C0
:10462000020C08BF4CEBD37C04E04FF0080C01E017
:104630004FEAD37C0CEB4C0526FA05F606F007068C
:10464000B6F1040C06D20EEB860CBDE870404CF0BF
:10465000010C6047DFE80CF0090B02024FF000414B
:104660004FF00000A1F5002170BD19461046012849
:1046700051EB010418BFD4F5001484BF002001F0F1
:10468000004170BD0808A0F500114FEA31017047E4
:1046900043004FEAD30C4FEA3C0C43401FBF400796
:1046A0000CF1605113F0FE4F70471CF0006F03D106
:1046B00000200CF0004170470CF0004343EA5070BA
:1046C00010B540EACC0000F026F900BF00000092CF
:1046D0004FEA0001FFF7D6BF4FF000414FF0000056
:1046E000A1F500217047000090EA010F48BF81F05A
:1046F000004100F16281421A3CBF801A89184FEADA
:10470000D0524FF07F4C1CEA410FA2EBD15318BF9F
:104710009CEA026F00F03B804FF0004C4CEA002016
:104720004CEA012121FA03FC10EB0C0C1ED202F121
:10473000FF325FEA1C2040EBC25038BF70471CF0CC
:104740007F0F4FEA400C18BFBCF17F4F38BF704756
:10475000C3F12003994008BF20F00100BCF17F4F56
:1047600038BF7047A0F1C04000F01BB94FEA3C00D1
:10477000000A40EBC25028BF1CF0FF0F4FEA400C6C
:10478000E6D018BFBCF17F4F38BF7047EAE79CEA1C
:10479000026F05D010EA5C0F08BF00F000407047C0
:1047A00010B500F0B8F800BF64FBBE3E41000B0E30
:1047B000D3F19E0208D950F400034FEA032323FAF1
:1047C00002F048BF4042704710B500F0A4F800BFA7
:1047D00049922480002070476FF0004282EA200056
:1047E0007047000010F0004148BF4042B0FA80F32B
:1047F00010FA03F2C3F19D030BD051EAC35101EB50
:104800001220530638BF704700F1010008BF20F0A6
:10481000010070474FF47F0C1CEAD0121EBF1CEA47
:10482000D11392EA0C0F93EA0C0F00F0478090EA44
:10483000010F48BF42F480724FF0004C4CEA002058
:104840004CEA012102EB0302A0FB0113A2F50002D6
:10485000002918BF43F001035B0028BF4FEA330370
:1048600042EB22425FEA132C4CEBC2502EBFBCEB52
:10487000436FB2F57C0F70474FEA036CBCF1004FF9
:1048800008BF20F00100B2F57C0F38BF70470BD590
:1048900082F0FF0212F5803FC8BF704700F1C040B0
:1048A000D8BF00F00040704700F5000C5FEA4C0CE8
:1048B00048BF7047B0F1C04000F073B890EA010FF4
:1048C0000CEAD11348BF42F48072624538BF634599
:1048D00004D280EA010000F00040704710B500F0FB
:1048E0001AF800BF8900013E00F007B800F009B8CF
:1048F0005FEA410C5FEA1C6C08D080EA010000F01E
:1049000050B85FEA400C5FEA1C6CF6D14FF00040F3
:10491000A0F5800070470EF1020E2EF0030E5EF837
:10492000044B244204D44FEA4102B2F17F4F11D824
:104930004FEA4003B3F17F4F0CD80ED14FEAD07C41
:10494000B2F17F4F0CEB4C0C0CF1020C08BF4CEB9E
:10495000D17C04E04FF0080C01E04FEAD17C0CEB75
:104960004C0324FA03F404F00704B4F1040C06D257
:104970000EEB840CBDE810404CF0010C6047DFE802
:104980000CF0070802024FF00040A0F5800010BDB7
:104990000846420018BFD2F1807288BF00F0004084
:1049A00010BDFF2141EAD050C005704790EA010FC9
:1049B00048BF81F000413FF59EAE421A04D882F014
:1049C0000042A0EB020011444FEAD0524FF07F4C5E
:1049D0001CEA410FA2EBD15318BF9CEA026F4AD0E8
:1049E0004FF0004C4CEA00204CEA012121FA03FC74
:1049F000B0EB0C0C0FD412F0FE0F36D05FEA4C0077
:104A00001DD5001240EBC25038BF70471CF03F0F5D
:104A100018BF70470BE0A2F101025FEA1C2040EBD7
:104A2000C25038BF70471CF07F0F18BF7047C3F1EA
:104A30002003994014BF401E20F0010070478008F9
:104A40004FEA122308BF7047B0FA80FCA2EB0C02B9
:104A5000CCF1280C60FA0CF093EA122F04BF00EBA3
:104A6000C25070474FEAC3707047130A5FEADC1008
:104A700008BF7047F6E79CEA026F04D010EA5C0FAB
:104A800008BF0020704710B5FFF745FF40DFF63E36
:104A900081F000407047FEF703BE000000000000F8
:104AA0000000002F000000000700070000147F1422
:104AB0007F1400242A7F2A12006264081323003620
:104AC0004955225000000503000000001C2241004F
:104AD000000041221C000014083E08140008083E93
:104AE0000808000000A0600000080808080800008E
:104AF00060600000002010080402003E5149453E5D
:104B00000000427F4000004261514946002141457A
:104B10004B31001814127F10002745454539003CE1
:104B20004A494930000171090503003649494936AF
:104B300000064949291E000036360000000056369E
:104B40000000000814224100001414141414000082
:104B50004122140800020151090600324959513E10
:104B6000007C1211127C007F49494936003E4141C8
:104B70004122007F4141221C007F49494941007F79
:104B800009090901003E4149497A007F0808087F68
:104B90000000417F4100002040413F01007F081498
:104BA0002241007F40404040007F020C027F007F96
:104BB0000408107F003E4141413E007F090909067B
:104BC000003E4151215E007F0919294600464949AE
:104BD00049310001017F0101003F4040403F001F7B
:104BE0002040201F003F4038403F006314081463FA
:104BF00000070870080700615149454300007F41E4
:104C0000410000552A552A55000041417F0000040B
:104C10000201020400404040404000000102040044
:104C2000002054545478007F4844443800384444A9
:104C3000442000384444487F003854545418000835
:104C40007E0901020018A4A4A47C007F0804047853
:104C50000000447D4000004080847D00007F1028DB
:104C600044000000417F4000007C04180478007C70
:104C70000804047800384444443800FC24242418F0
:104C80000018242418FC007C08040408004854542C
:104C9000542000043F444020003C4040207C001C45
:104CA0002040201C003C4030403C00442810284458
:104CB000001CA0A0A07C004464544C4414141414A0
:104CC00014140000000000000000000000000000BC
:104CD0000000000000F80000000000000033300079
:104CE000000000100C06100C060000000000000080
:104CF000000040C07840C0784000043F04043F04F6
:104D00000400007088FC08300000001820FF211EFD
:104D10000000F008F000E018000000211C031E2134
:104D20001E0000F00888700000001E2123241927AF
:104D3000211010160E00000000000000000000000E
:104D40000000000000E01804020000000007182026
:104D5000400000020418E000000000402018070096
:104D60000000404080F0804040000202010F01023C
:104D70000200000000F0000000000101011F01011D
:104D80000100000000000000000080B07000000082
:104D9000000000000000000000000001010101010E
:104DA00001010000000000000000003030000000A1
:104DB0000000000000008060180400601806010078
:104DC000000000E010080810E000000F1020201084
:104DD0000F00001010F8000000000020203F2020ED
:104DE0000000007008080888700000302824222184
:104DF000300000300888884830000018202020113A
:104E00000E000000C02010F8000000070424243F1A
:104E1000240000F8088888080800001921202011C3
:104E20000E0000E0108888180000000F11202011EB
:104E30000E0000380808C83808000000003F0000D5
:104E400000000070880808887000001C22212122C0
:104E50001C0000E010080810E000000031222211C0
:104E60000F00000000C0C000000000000030300053
:104E700000000000008000000000000080600000D2
:104E8000000000008040201008000001020408100B
:104E9000200040404040404040000404040404041A
:104EA00004000008102040800000002010080402C8
:104EB0000100007048080808F000000000303601CA
:104EC0000000C030C828E810E00007182724231489
:104ED0000B000000C038E0000000203C2302022745
:104EE000382008F8888888700000203F2020201192
:104EF0000E00C030080808083800071820202010CD
:104F0000080008F808080810E000203F20202010C2
:104F10000F0008F88888E8081000203F2020232090
:104F2000180008F88888E8081000203F20000300D7
:104F30000000C03008080838000007182020221E92
:104F4000020008F808000008F808203F21010121AC
:104F50003F20000808F8080800000020203F20201B
:104F6000000000000808F8080800C08080807F006A
:104F7000000008F888C028180800203F20012638C3
:104F8000200008F8080000000000203F202020201A
:104F9000300008F8F800F8F80800203F003F003F14
:104FA000200008F830C00008F808203F200007184B
:104FB0003F00E01008080810E0000F10202020102B
:104FC0000F0008F808080808F000203F210101013F
:104FD0000000E01008080810E0000F1824243850E2
:104FE0004F0008F8888888887000203F2000030C54
:104FF000302000708808080838000038202121225D
:105000001C00180808F8080818000000203F2000BD
:10501000000008F808000008F808001F20202020E1
:105020001F000878880000C83808000007380E0103
:105030000000F80800F80008F800033C0700073CEF
:105040000300081868808068180820302C03032C9F
:1050500030200838C800C83808000000203F200071
:10506000000010080808C838080020382621202031
:105070001800000000FE020202000000007F404015
:105080004000000C30C000000000000000010638A5
:10509000C00000020202FE000000004040407F000D
:1050A00000000000040202020400000000000000F2
:1050B00000000000000000000000808080808080F0
:1050C00080800002020400000000000000000000D8
:1050D000000000008080808000000019242222222D
:1050E0003F2008F8008080000000003F11202011C0
:1050F0000E000000008080800000000E11202020A3
:105100001100000000808088F800000E112020109F
:105110003F200000808080800000001F2222222289
:105120001300008080F0888888180020203F20200D
:1051300000000000808080808000006B9494949335
:10514000600008F8008080800000203F21000020DF
:105150003F2000809898000000000020203F202081
:105160000000000000809898000000C08080807FD0
:10517000000008F8000080808000203F24022D30CD
:105180002000000808F8000000000020203F202038
:1051900000008080808080808000203F20003F20B1
:1051A000003F8080008080800000203F21000020A0
:1051B0003F200000808080800000001F20202020F1
:1051C0001F00808000808000000080FFA12020114F
:1051D0000E000000008080808000000E112020A0C2
:1051E000FF80808080008080800020203F21200080
:1051F000010000008080808080000033242424246B
:105200001900008080E0808000000000001F202046
:1052100000008080000000808000001F20202010FF
:105220003F20808080000080808000010E300806D2
:10523000010080800080008080800F300C030C30E3
:105240000F0000808000808080000020312E0E3111
:105250002000808080000080808080818E70180611
:10526000010000808080808080000021302C22217D
:10527000300000000000807C020200000000003FBF
:10528000404000000000FF00000000000000FF00A0
:1052900000000002027C800000000040403F00004F
:1052A00000000006010102020404000000000000EA
:1052B0000000000002400000000000A0000000000C
:1052C00005400000000000C8000000000C40000085
:1052D0000000409C00000000194000000020BCBEFF
:1052E0000000000034400000BFC91B8E0000000415
:1052F000B5400000504BCFD06607E2CF0100000060
:105300006C4100003E8251AADFEEA734010000008C
:10531000D9420000DCB5A0E23A301F97FFFFFFFF43
:10532000B4450000FD25A0C8E9A3C14FFFFFFFFF62
:10533000FF3F00000000008000000000FF3F000071
:1053400000000080000000008453000800000020DE
:105350009C0200006C010008885400089C02002098
:10536000A4060000C80100081C0000004300000063
:10537000F8FFFFFF0C0000000E0000000F0000000F
:105380002E0000001184A24A0468090102030406E9
:105390000708090C6910051402040608154040426C
:1053A000CC000B1440A09E8282829EA02020000D83
:1053B000113F908840432C1028464180801C100CDF
:1053C00044012B45C606041144140C3809804020C2
:1053D0001E2040407F20031240403809088848289A
:1053E000180FE8080109111F2B0809013AFF0609E7
:1053F000112139C0080A1204F49494FF9494F4041F
:10540000E1080D10201F20484442415F41424448BA
:105410008029764C88780F7F0911601E201048463D
:1054200041012A7F050911C029350B18C838402EC3
:1054300008040201FF3C19010213FF080E12C8B84C
:105440008FE888C820900C030C902060161808FF85
:1054500004041A3FC204144040702809FC24242488
:10546000FC2526240802110400101140308F80848E
:105470004C55252525554C80808000092C9A99197A
:085480003FCDCCCC3D022B46D0
:0400000508000131BD
:00000001FF
